:1000000042C0ADC15BC05AC059C058C057C056C0ED
:1000100055C054C053C052C051C050C04FC04EC054
:100020004DC04CC04BC04AC049C048C047C046C084
:1000300045C044C0040309041C037700770077001F
:100040002E00660069007300630068006C002E00DB
:10005000640065000E035500530042006100730008
:10006000700012011001FF000008C016DC0503013A
:1000700001020001090212000101008019090400B7
:1000800000000000000011241FBECFEFD4E0DEBF4F
:10009000CDBF11E0A0E0B1E0E6E2FFE002C00590D4
:1000A0000D92A230B107D9F711E0A2E0B1E001C092
:1000B0001D92A734B107E1F7C8D433C7A1CFE9E651
:1000C000F0E0808183608083E89A08951F93CF9346
:1000D000DF9360912801635067FD13C08091250173
:1000E000CCE0D0E0C81BD109C45DDE4F8091240173
:1000F0008D3209F462C08091020187FD84C01092A4
:1001000028018091000184FF4AC0609101016F3F86
:1001100009F445C0693070F1685060930101809125
:10012000180198E889278093180168E080910201FE
:1001300087FD8BC0209126013091270186FF6DC07D
:10014000A9E1B1E080E090E0F901E80FF91FE49146
:10015000ED9301966817C1F76150862F90E06F5FAD
:100160000196820F931F9093270180932601162FEB
:100170001C5F0BC0109201018091180198E889273B
:1001800080931801662391F614E089E191E0E3D0B1
:100190001C3019F08FEF809301011093000194E15E
:1001A00083B1837031F49150D9F7109229011092E4
:1001B0002301DF91CF911F910895683009F09FCFFF
:1001C00083EC809318018AE580930001109202016C
:1001D0008881807659F59A8110922101898188233E
:1001E00009F043C01092220122E081E291E0909355
:1001F0002701809326018F81882319F49E8192170D
:1002000008F1922F1FC0CE0131D48F3F51F18823C6
:1002100009F475CF1092010172CF962FD901E9E14F
:10022000F1E08D9181939150E1F796CFCE0110D5F9
:10023000282F8F3F01F7888187FD25C09FEF80E839
:1002400080930201909301015ACF89E191E0B0D4EB
:10025000682F893008F453C08FEF809301011EE1AD
:100260009CCF8EE1809300014ACF853071F08630BB
:1002700091F0883031F1893061F18A3031F120E03C
:1002800081E291E0B4CF9E81DACF9093290120E002
:1002900081E291E0ACCF8B81813049F18230F9F07D
:1002A000833029F020E080E480930201A4CF9923D9
:1002B00049F584E390E0909327018093260124E0A0
:1002C000F2CF21E08BE291E092CF21E081E291E058
:1002D0008ECF90932B0120E081E291E088CF84E7DC
:1002E00090E0909327018093260122E1DCCF82E603
:1002F00090E0909327018093260122E1D4CF182F1C
:100300001C5F43CF913051F0923061F684E590E06C
:1003100090932701809326012EE0C5CF88E390E0DB
:1003200090932701809326012CE1BDCFA82FB92FF0
:1003300080E090E041E050EA60956F5F58F42D91C5
:1003400038EF82279795879510F0842795273F5F90
:10035000C8F3F3CF0895EADF8D939D930895CF936B
:10036000CFB7CF93C395189BE9F7189B09C0189B8B
:1003700007C0189B05C0189B03C0189B01C0A1C0F3
:10038000DF93C0912501DD27C45DDE4F189B02C0BD
:10039000DF91EBCF2F930F931F9303B12FEF00FB50
:1003A00020F94F933F9313B14FEF012700FB21F941
:1003B0003BE031C04E7F012F13B1216028C0102FC8
:1003C0004D7F2260000003B129C04B7F2460012FC4
:1003D000000013B12BC013B1477F28602AC04F7EA5
:1003E00003B120612CC04F7D13B120622FC04F7B21
:1003F00003B1206432C0422703B149934FEF00009C
:10040000102710FB20F913B11370C9F1297F91F265
:10041000012700FB21F903B1237F89F2315058F104
:10042000102710FB22F913B1277E79F2012700FB78
:1004300023F92F7C81F203B1102710FB24F92F79C7
:1004400071F200C013B1012700FB25F92F7359F297
:1004500000C003B1102710FB26F9223040F200C083
:1004600013B1012700FB27F9243028F64F772068C5
:1004700013B10000F9CF11E01CBB002717C03B509F
:100480003195C31BD04011E01CBB0881033CE9F04F
:100490000B34D9F0209123011981110F1213EDCFE4
:1004A000093641F10D3211F0013E39F700932A016E
:1004B0003F914F911F910F912F91DF91CCB3C0FDD0
:1004C00051CFCF91CFBFCF91189520912A012223F0
:1004D00079F310912801112311F5343012F1309382
:1004E000280120932401109125013BE0311B30931A
:1004F000250117C00091280101308CF40AE53091E4
:10050000000134FD10C000930001C8E1D1E00FC02C
:100510002795A8F45150A9F4220F0000F9CF4AE51D
:1005200003C042ED01C0432FC4E1D0E032E014B17A
:100530001360289A14B905B120E413E05F930127F2
:1005400056E005B9279520F4515021F4220FF9CF38
:10055000012756E000003B5A05B9D0F2279528F450
:10056000515029F4220F0000F9CF012756E02795BA
:1005700005B920F4515021F4220FF9CF012756E09C
:100580002991332305B921F60C7F10912901110F10
:10059000C651D04005B911F01093230111E01CBBE6
:1005A000016014B11C7F402F4C7F5F9100C000C0E0
:1005B00005B914B945B97CCF809145018CBD8091B6
:1005C00042018DBD0895282F8823A1F0883008F0BE
:1005D0003FC080E893E0909344018093430124302E
:1005E00001F12530A0F0263081F1263050F127307E
:1005F000E1F0089581EA93E09093440180934301F0
:1006000082E58093450181E0809342010895223084
:10061000A1F0233070F4213061F780EC8093460123
:10062000089588E180934601089583E08093460110
:10063000089580E380934601089580E68093460103
:1006400008958CE080934601089520934601089513
:1006500081EA93E090934401809343011092420118
:10066000293041F02A3050F4283051F683E5809348
:100670004501089582E58093450108952B3031F0BE
:100680002C3009F0BDCF81E08093420181E5809359
:100690004501089526B59091460186B5821B8917BC
:1006A000E0F308952C9A3D9A459884B18C6284B900
:1006B0002A982D9896B52091460186B5891B8217F8
:1006C000E0F32A9A96B586B5891B8217E0F32A983B
:1006D0008091430190914401815A934009F008951B
:1006E000809145018CBD809142018DBD089584B1FA
:1006F000837D84B985B1837D85B93D981CBC0895FF
:10070000582F2091460140E030E057FD16C02B984D
:10071000440F1C994F5F2D9A96B586B5891B821799
:10072000E0F32D9896B586B5891B8217E0F33F5FFD
:10073000383029F0550F57FFEACF2B9AE9CF842F95
:1007400008958EBD0DB407FEFDCF8EB508950F93AD
:100750001F930FE1E0914301F09144018CEA099568
:10076000E0914301F091440183E50995E091430153
:10077000F091440180E00995182FE0914301F09138
:10078000440180E00995133539F11CBC96B52091E0
:10079000460186B5891B8217E0F32D9A96B586B57A
:1007A000891B8217E0F32D98E0914301F0914401F9
:1007B00083E0E13AF80721F0002351F00150CECF59
:1007C000809145018CBD809142018DBD0023B1F720
:1007D00081E01F910F91089580E01F910F9108957E
:1007E000EF92FF920F931F937B018C01862F8170F4
:1007F000880F880F880FE0914301F09144018062D7
:100800000995D801C70129E0B695A79597958795D1
:100810002A95D1F7E0914301F0914401099516958D
:100820000795F794E794E0914301F09144018E2DF0
:100830000995E0914301F091440180E009951F91F1
:100840000F91FF90EF9008950F931F938C01E0910B
:100850004301F091440180EA0995E0914301F09150
:100860004401812F0995E0914301F0914401802FCB
:100870000995E0914301F091440180E009951F91B1
:100880000F910895FF920F931F938C01F62EE09124
:100890004301F091440180EC0995E0914301F0910E
:1008A0004401812F0995E0914301F0914401802F8B
:1008B0000995E0914301F09144018F2D09958EE156
:1008C000B7D080E01F910F91FF900895CF92DF92F3
:1008D000EF92FF920F931F936B017C01142FE09115
:1008E0004301F09144018CE40995D701C60149E028
:1008F000B695A795979587954A95D1F7E0914301CD
:10090000F09144010995D701C601B695A795979531
:100910008795E0914301F09144010995E0914301ED
:10092000F091440180E009951F3FF1F016B50EE10A
:10093000C701B60155DF8F3F79F486B5811B8D3332
:10094000B8F316B50150A1F781E01F910F91FF9008
:10095000EF90DF90CF90089580E01F910F91FF906E
:10096000EF90DF90CF9008958FE062D080E01F91EC
:100970000F91FF90EF90DF90CF900895CF92DF928C
:10098000EF92FF920F931F936B017C01042F122FA4
:10099000862F8170880F880F880FE0914301F091B6
:1009A000440180640995D701C60169E0B695A79511
:1009B000979587956A95D1F7E0914301F0914401AD
:1009C0000995D701C601B695A79597958795E091AA
:1009D0004301F09144010995E0914301F0914401F4
:1009E000802F09951123C1F00F37F1F016B50EE1F4
:1009F000C701B601F5DE8F3779F486B5811B8D33DB
:100A0000B8F316B50150A1F781E01F910F91FF9047
:100A1000EF90DF90CF90089580E01F910F91FF90AD
:100A2000EF90DF90CF9008958FE002D080E0F5CF77
:100A3000382F882349F020E096B586B5891B8C3382
:100A4000E0F32F5F2317C0F308951BB815B88BEFA1
:100A50008AB98FEF84B914B893E097B98EEF88B94B
:100A600095BD2DDB789432DB31DBFDCFFF920F9308
:100A70001F93CF93DF93F82E292F062F4091030168
:100A8000413051F0443041F01FEF812FDF91CF9181
:100A90001F910F91FF900895002309F487C08F2DB7
:100AA000922F9C01E90110E053C0809114019091B4
:100AB0001501892B09F058C0609110017091110146
:100AC000809112019091130121E0488157DF8091BC
:100AD0000401909105010197909305018093040111
:100AE000892BD9F4109203018091160181FF3AC03D
:100AF0008091170190E02091140130911501821727
:100B0000930781F1609110017091110180911201A0
:100B1000909113014881DADE11E0809110019091EB
:100B20001101A0911201B09113010196A11DB11DF7
:100B30008093100190931101A0931201B0931301BF
:100B400021969E012F19201708F09FCF4091030195
:100B5000413009F4AACF6881809110019091110170
:100B600091DEB5CF11E0D9CF6091100170911101E4
:100B7000809112019091130120E04881FFDE809165
:100B80001701815080931701882309F0A0CF60914D
:100B9000100170911101809112019091130148810F
:100BA00095DE809114018093170191CF10E06DCFF5
:100BB0000F931F93CF93DF93082F162F40910301BC
:100BC000842F8250823038F01FEF812FDF91CF9138
:100BD0001F910F910895662399F1802F9C01E901DF
:100BE00020C080911001909111012EDE88838091A8
:100BF000100190911101A0911201B0911301019681
:100C0000A11DB11D8093100190931101A0931201B9
:100C1000B093130121969E01201B211778F4409177
:100C200003014230F1F66091100170911101809141
:100C3000120190911301D4DD8883D9CF183028F6A2
:100C400010920301812FDF91CF911F910F91089591
:100C50000F931F93CF93DF938C01EC018981813037
:100C6000F1F0823009F4BCC0833091F1843009F492
:100C70008EC0873009F462C0853009F42DC18630FA
:100C800009F4E6C0883009F4B4C0893009F42BC1F6
:100C90008A3009F43CC180E0C8E0D1E043C03B9811
:100CA000439A00000000339BA1C03A9A429800008A
:100CB0000000339B40C08091060185DC3A98429A3F
:100CC000109207014198EEDC80E0C8E0D1E02AC034
:100CD000E0914301F0914401E8018A810995C8E05F
:100CE000D1E0809308012091430130914401F80143
:100CF0008381F90109958093090120914301309185
:100D00004401F8018481F901099580930A01209139
:100D1000430130914401F8018581F90109958093DF
:100D20000B0184E0D0932701C0932601DF91CF917E
:100D30001F910F91089588E046DCC0CF8091070194
:100D4000882399F4E8019B8180E02A8130E0822B9E
:100D5000932BAA2797FDA095BA2F8093100190930B
:100D60001101A0931201B0931301F801978180E063
:100D7000268130E0822B932B909305018093040110
:100D800083E0809303018FEFC8E0D1E0CBCF809167
:100D90000701882399F4E8019B8180E02A8130E0F3
:100DA000822B932BAA2797FDA095BA2F8093100131
:100DB00090931101A0931201B0931301F801978150
:100DC00080E0268130E0822B932B90930501809365
:100DD000040182E0809303018FEFC8E0D1E0A2CF4D
:100DE00086DC419A80E0C8E0D1E09CCF89E0EBDB73
:100DF00067CF80910701882399F4F801938180E0FF
:100E0000228130E0822B932BAA2797FDA095BA2F41
:100E10008093100190931101A0931201B0931301DC
:100E2000109215011092140110921601E8019F8191
:100E300080E02E8130E0822B932B909305018093EC
:100E4000040184E0809303018FEFC8E0D1E06ACF12
:100E500080910701882399F4E8019B8180E02A8131
:100E600030E0822B932BAA2797FDA095BA2F809371
:100E7000100190931101A0931201B0931301F80196
:100E800084819581292F2F7020931601492F50E0DE
:100E9000407F507042955295507F5427407F542791
:100EA000480F511D509315014093140120FF02C0BB
:100EB00040931701E8019F8180E02E8130E0822B72
:100EC000932B909305018093040181E080930301AB
:100ED0008FEFC8E0D1E026CF3ADCC8E0D1E08093C4
:100EE000080181E01FCF81E080930701F801828132
:100EF0009381A481B5818093100190931101A093F7
:100F00001201B093130180E0C8E0D1E00BCFE801FB
:100F10008A8180930601C8E0D1E01092080181E047
:060F200001CFF894FFCFA1
:020F26005AFF70
:00000001FF
